******************************************************************************
               TMS320C6x Linker PC v7.4.1                      
******************************************************************************
>> Linked Sat Jan 26 16:39:07 2013

OUTPUT FILE NAME:   <Memory_Sharing.out>
ENTRY POINT SYMBOL: "_c_int00"  address: 00810820


MEMORY CONFIGURATION

         name            origin    length      used     unused   attr    fill
----------------------  --------  ---------  --------  --------  ----  --------
  VECTORS               00800000   00000200  00000200  00000000  RWIX
  LL2                   00800200   0001ee00  00014cc2  0000a13e  RWIX
  C0L2                  1081f000   00001000  00000484  00000b7c  RWIX


SEGMENT ALLOCATION MAP

run origin  load origin   length   init length attrs members
----------  ----------- ---------- ----------- ----- -------
00800000    00800000    0001284e   0001284e    r-x
  00800000    00800000    00000200   00000200    r-x vecs
  00800200    00800200    00010c40   00010c40    r-x .text
  00810e40    00810e40    00001a0e   00001a0e    r-- .const
00812850    00812850    00001800   00000000    rw-
  00812850    00812850    00001000   00000000    rw- .stack
  00813850    00813850    00000800   00000000    rw- .sysmem
00814050    00814050    00000840   00000720    rw-
  00814050    00814050    00000550   00000550    rw- .fardata
  008145a0    008145a0    000001d0   000001d0    rw- .far
  00814770    00814770    00000120   00000000    rw- .cio
00814890    00814890    000000f4   000000d8    rw-
  00814890    00814890    000000d8   000000d8    rw- .neardata
  00814968    00814968    0000001c   00000000    rw- .bss
00814984    00814984    00000540   00000540    r--
  00814984    00814984    00000540   00000540    r-- .cinit
1081f000    1081f000    00000484   00000484    rw-
  1081f000    1081f000    00000484   00000484    rw- GlobalData


SECTION ALLOCATION MAP

 output                                  attributes/
section   page    origin      length       input sections
--------  ----  ----------  ----------   ----------------
vecs       0    00800000    00000200     
                  00800000    00000200     MEM_share_vectors.obj (vecs)

.text      0    00800200    00010c40     
                  00800200    00005ac0     KeyStone_common.obj (.text)
                  00805cc0    000023e0     KeyStone_DDR_Init.obj (.text)
                  008080a0    00000b40     MEM_sharing.obj (.text)
                  00808be0    00000660     MEM_sharing.obj (.text:retain)
                  00809240    000005c0     rts6600_elf.lib : divd.obj (.text:__c6xabi_divd)
                  00809800    000005c0                     : _printfi.obj (.text:_getarg_diouxp)
                  00809dc0    00000520     KeyStone_common.obj (.text:Core_MPAX)
                  0080a2e0    00000520     MEM_share_DSP_core.obj (.text)
                  0080a800    000004e0     KeyStone_common.obj (.text:retain)
                  0080ace0    00000460     rts6600_elf.lib : _printfi.obj (.text:_printfi)
                  0080b140    00000460                     : _printfi.obj (.text:_setfield)
                  0080b5a0    000003c0     MEM_share_Edma_Share.obj (.text:retain)
                  0080b960    000003a0     rts6600_elf.lib : fputs.obj (.text:fputs)
                  0080bd00    00000320                     : _printfi.obj (.text:_pproc_fge)
                  0080c020    000002e0                     : _printfi.obj (.text:_pproc_fwp)
                  0080c300    000002c0     MEM_share_Edma_Share.obj (.text)
                  0080c5c0    000002a0     rts6600_elf.lib : _printfi.obj (.text:fcvt)
                  0080c860    00000280                     : divf.obj (.text:__c6xabi_divf)
                  0080cae0    00000280                     : _printfi.obj (.text:ecvt)
                  0080cd60    00000280                     : memory.obj (.text:free)
                  0080cfe0    00000240                     : imath64.obj (.text:__c6xabi_divull)
                  0080d220    00000240                     : _printfi.obj (.text:_pconv_e)
                  0080d460    00000240                     : _printfi.obj (.text:_pproc_diouxp)
                  0080d6a0    00000220                     : _printfi.obj (.text:_pproc_str)
                  0080d8c0    00000220                     : fputc.obj (.text:fputc)
                  0080dae0    00000200                     : _printfi.obj (.text:_pconv_g)
                  0080dce0    00000200                     : setvbuf.obj (.text:setvbuf)
                  0080dee0    000001c0                     : _printfi.obj (.text:_mcpy)
                  0080e0a0    000001a0                     : trgdrv.obj (.text:HOSTrename)
                  0080e240    000001a0     MEM_share_EDMA_Timer_Intc_setup.obj (.text)
                  0080e3e0    000001a0     rts6600_elf.lib : imath40.obj (.text:__c6xabi_divul)
                  0080e580    00000180                     : copy_decompress_rle.obj (.text:__TI_decompress_rle_core)
                  0080e700    00000180                     : memory.obj (.text:malloc)
                  0080e880    00000140                     : _printfi.obj (.text:_pproc_fflags)
                  0080e9c0    00000140                     : lowlev.obj (.text:getdevice)
                  0080eb00    00000120                     : fclose.obj (.text:_closefile)
                  0080ec20    00000120                     : _printfi.obj (.text:_ltostr)
                  0080ed40    00000120                     : fseek.obj (.text:fseek)
                  0080ee60    00000100                     : trgdrv.obj (.text:HOSTlseek)
                  0080ef60    00000100                     : autoinit.obj (.text:_auto_init_elf)
                  0080f060    00000100                     : _io_perm.obj (.text:_wrt_ok)
                  0080f160    00000100                     : cpy_tbl.obj (.text:copy_in)
                  0080f260    000000e0                     : trgdrv.obj (.text:HOSTopen)
                  0080f340    000000e0                     : _printfi.obj (.text:_div)
                  0080f420    000000e0                     : atoi.obj (.text:atoi)
                  0080f500    000000e0                     : lowlev.obj (.text:close)
                  0080f5e0    000000e0                     : copy_zero_init.obj (.text:decompress:ZI:__TI_zero_init)
                  0080f6c0    000000e0                     : ltoa.obj (.text:ltoa)
                  0080f7a0    000000e0                     : memset.obj (.text:memset)
                  0080f880    000000e0                     : printf.obj (.text:printf)
                  0080f960    000000c0                     : trgdrv.obj (.text:HOSTread)
                  0080fa20    000000c0                     : trgdrv.obj (.text:HOSTunlink)
                  0080fae0    000000c0                     : trgdrv.obj (.text:HOSTwrite)
                  0080fba0    000000c0                     : divu.obj (.text:__divu)
                  0080fc60    000000c0                     : fflush.obj (.text:_doflush)
                  0080fd20    000000c0                     : exit.obj (.text:exit)
                  0080fde0    000000c0                     : tls.obj (.text:tls:init:__TI_tls_init)
                  0080fea0    000000a0                     : trgdrv.obj (.text:HOSTclose)
                  0080ff40    000000a0                     : fopen.obj (.text:_cleanup)
                  0080ffe0    000000a0                     : _printfi.obj (.text:_ecpy)
                  00810080    000000a0                     : _printfi.obj (.text:_fcpy)
                  00810120    000000a0                     : memory.obj (.text:_minit)
                  008101c0    000000a0                     : _printfi.obj (.text:_pconv_f)
                  00810260    000000a0                     : lowlev.obj (.text:finddevice)
                  00810300    000000a0                     : lowlev.obj (.text:lseek)
                  008103a0    000000a0                     : memcpy64.obj (.text:memcpy)
                  00810440    000000a0                     : memory.obj (.text:minsert)
                  008104e0    000000a0                     : memory.obj (.text:mremove)
                  00810580    000000a0                     : lowlev.obj (.text:write)
                  00810620    00000080     MEM_share_MemCopy8.obj (.text)
                  008106a0    00000080     rts6600_elf.lib : fixdu.obj (.text:__c6xabi_fixdu)
                  00810720    00000080                     : fixfu.obj (.text:__c6xabi_fixfu)
                  008107a0    00000080                     : llshift.obj (.text:__c6xabi_llshl)
                  00810820    00000080                     : boot.obj (.text:_c_int00)
                  008108a0    00000080                     : trgmsg.obj (.text:readmsg)
                  00810920    00000080                     : lowlev.obj (.text:unlink)
                  008109a0    00000060                     : cpp_init.obj (.text:__TI_cpp_init)
                  00810a00    00000060                     : frcmpyd_div.obj (.text:__c6xabi_frcmpyd_div)
                  00810a60    00000060                     : llshift.obj (.text:__c6xabi_llshru)
                  00810ac0    00000060                     : imath64.obj (.text:_subcull)
                  00810b20    00000060                     : memccpy.obj (.text:memccpy)
                  00810b80    00000060                     : trgmsg.obj (.text:writemsg)
                  00810be0    00000040     MEM_share_vectors.obj (.text)
                  00810c20    00000040     rts6600_elf.lib : isinf.obj (.text:__c6xabi_isinf)
                  00810c60    00000040                     : _printfi.obj (.text:__c6xabi_isnan)
                  00810ca0    00000040                     : strasg.obj (.text:__strasgi_64plus)
                  00810ce0    00000040                     : args_main.obj (.text:_args_main)
                  00810d20    00000040                     : fputs.obj (.text:puts)
                  00810d60    00000020                     : negll.obj (.text:__c6xabi_negll)
                  00810d80    00000020                     : _lock.obj (.text:_nop)
                  00810da0    00000020                     : printf.obj (.text:_outc)
                  00810dc0    00000020                     : printf.obj (.text:_outs)
                  00810de0    00000020                     : exit.obj (.text:abort)
                  00810e00    00000020                     : copy_decompress_none.obj (.text:decompress:none:__TI_decompress_none)
                  00810e20    00000020                     : copy_decompress_rle.obj (.text:decompress:rle24:__TI_decompress_rle24)

.const     0    00810e40    00001a0e     
                  00810e40    00001628     KeyStone_common.obj (.const:.string)
                  00812468    000001cb     MEM_sharing.obj (.const:.string)
                  00812633    00000002     rts6600_elf.lib : fputs.obj (.const:.string)
                  00812635    00000003     --HOLE-- [fill = 0]
                  00812638    00000101                     : ctype.obj (.const:.string:_ctypes_)
                  00812739    000000c2     KeyStone_DDR_Init.obj (.const:.string)
                  008127fb    00000023     rts6600_elf.lib : _printfi.obj (.const:.string)
                  0081281e    00000018     MEM_share_EDMA_Timer_Intc_setup.obj (.const:.string)
                  00812836    00000018     MEM_share_Edma_Share.obj (.const:.string)

.stack     0    00812850    00001000     UNINITIALIZED
                  00812850    00000008     rts6600_elf.lib : boot.obj (.stack)
                  00812858    00000ff8     --HOLE--

.sysmem    0    00813850    00000800     UNINITIALIZED
                  00813850    00000008     rts6600_elf.lib : memory.obj (.sysmem)
                  00813858    000007f8     --HOLE--

.fardata   0    00814050    00000550     
                  00814050    000001e0     rts6600_elf.lib : defs.obj (.fardata:_ftable)
                  00814230    000000a0                     : lowlev.obj (.fardata:_stream)
                  008142d0    00000078                     : lowlev.obj (.fardata:_device)
                  00814348    00000060     MEM_sharing.obj (.fardata:testCases)
                  008143a8    0000004c     MEM_sharing.obj (.fardata:dmaEnableMaskPattern)
                  008143f4    00000004     rts6600_elf.lib : defs.obj (.fardata)
                  008143f8    00000040     KeyStone_common.obj (.fardata:gstruMpuAddrRange)
                  00814438    00000028     KeyStone_common.obj (.fardata:gEDMA_TC_Regs)
                  00814460    00000024     KeyStone_common.obj (.fardata:internal_exception_str)
                  00814484    00000004     --HOLE--
                  00814488    00000024     KeyStone_common.obj (.fardata:timerRegs)
                  008144ac    00000004     --HOLE--
                  008144b0    00000020     KeyStone_common.obj (.fardata:MPU_Regs)
                  008144d0    00000020     KeyStone_common.obj (.fardata:bus_err_stat_str)
                  008144f0    00000020     KeyStone_common.obj (.fardata:gCIC_EXC_EN_MASK)
                  00814510    0000001c     MEM_sharing.obj (.fardata:coreEnableMaskPattern)
                  0081452c    00000004     --HOLE--
                  00814530    00000018     KeyStone_common.obj (.fardata:Peri_MPU_err_type_str)
                  00814548    0000000c     MEM_share_Edma_Share.obj (.fardata:edma_sys_event_num)
                  00814554    00000004     --HOLE--
                  00814558    0000000c     KeyStone_common.obj (.fardata:gEDMACCRegs)
                  00814564    00000004     --HOLE--
                  00814568    0000000c     MEM_sharing.obj (.fardata:priorityPattern)
                  00814574    0000000c     rts6600_elf.lib : exit.obj (.fardata)
                  00814580    0000000c                     : memory.obj (.fardata)
                  0081458c    00000004     --HOLE--
                  00814590    00000008     KeyStone_common.obj (.fardata:Ns_str)
                  00814598    00000008     rts6600_elf.lib : _lock.obj (.fardata)

.far       0    008145a0    000001d0     
                  008145a0    00000140     rts6600_elf.lib : defs.obj (.far) [fill = 0]
                  008146e0    00000068     KeyStone_common.obj (.far) [fill = 0]
                  00814748    00000010     KeyStone_common.obj (.far:Core_MPAX)
                  00814758    0000000c     MEM_share_EDMA_Timer_Intc_setup.obj (.far) [fill = 0]
                  00814764    00000004     --HOLE--
                  00814768    00000008     rts6600_elf.lib : trgdrv.obj (.far) [fill = 0]

.cio       0    00814770    00000120     UNINITIALIZED
                  00814770    00000120     rts6600_elf.lib : trgmsg.obj (.cio)

.neardata 
*          0    00814890    000000d8     
                  00814890    000000b8     KeyStone_common.obj (.neardata)
                  00814948    00000014     MEM_sharing.obj (.neardata)
                  0081495c    0000000c     MEM_share_Edma_Share.obj (.neardata)

.rodata    0    00814968    00000000     UNINITIALIZED

.bss       0    00814968    0000001c     UNINITIALIZED
                  00814968    0000001c     MEM_share_DSP_core.obj (.bss)

.cinit     0    00814984    00000540     
                  00814984    0000025c     (.cinit..fardata.load) [load image, compression = rle]
                  00814be0    000001cd     (.cinit.GlobalData.load) [load image, compression = rle]
                  00814dad    00000003     --HOLE-- [fill = 0]
                  00814db0    000000bc     (.cinit..neardata.load) [load image, compression = rle]
                  00814e6c    0000001a     (.cinit..far.load) [load image, compression = rle]
                  00814e86    00000002     --HOLE-- [fill = 0]
                  00814e88    0000000c     (__TI_handler_table)
                  00814e94    00000008     (.cinit..bss.load) [load image, compression = zero_init]
                  00814e9c    00000028     (__TI_cinit_table)

GlobalData 
*          0    1081f000    00000484     
                  1081f000    00000484     MEM_sharing.obj (GlobalData)


LINKER GENERATED COPY TABLES

__TI_cinit_table @ 00814e9c records: 5, size/record: 8, table size: 40
	.fardata: load addr=00814984, load size=0000025c bytes, run addr=00814050, run size=00000550 bytes, compression=rle
	GlobalData: load addr=00814be0, load size=000001cd bytes, run addr=1081f000, run size=00000484 bytes, compression=rle
	.neardata: load addr=00814db0, load size=000000bc bytes, run addr=00814890, run size=000000d8 bytes, compression=rle
	.far: load addr=00814e6c, load size=0000001a bytes, run addr=008145a0, run size=000001d0 bytes, compression=rle
	.bss: load addr=00814e94, load size=00000008 bytes, run addr=00814968, run size=0000001c bytes, compression=zero_init


LINKER GENERATED HANDLER TABLE

__TI_handler_table @ 00814e88 records: 3, size/record: 4, table size: 12
	index: 0, handler: __TI_decompress_rle24
	index: 1, handler: __TI_decompress_none
	index: 2, handler: __TI_zero_init


GLOBAL SYMBOLS: SORTED ALPHABETICALLY BY Name 

address    name
--------   ----
008051ec   Bus_error_handler
00810de0   C$$EXIT
00810bd8   C$$IO$$
00806824   C6670_EVM_DDR_Init
00806da4   C6678_EVM_DDR_Init
00814894   CGEM_regs
008148b8   CIC_Regs
0080e2a0   CP_INTC_Init_EDMA
00808584   ConfigureTest
00807c80   DDR_Address_Test
00807ac0   DDR_Fill_Test
008148ac   DDR_Regs
00814924   DSP_Core_Clock_KHz
0080a74c   DSP_Core_Test_Start
0080a2e0   DSP_core_mem_share_Test
00807360   Dual_Nyquist_EVM_DDR_Init
008041e4   EDMA_CC_error_handler
0080b5a0   EDMA_ISR
00804420   EDMA_TC_error_handler
0080e240   EDMA_Timer_Interrupts_Init
00805be0   EDMA_copy
008045c8   EDMA_error_handler
00808410   EDMA_init_for_mem_share
0080880c   EDMA_pri_set
00805b54   EDMA_wait
00805b44   EXC_NMI
00805a34   EXC_internal
00805a24   EXC_swgen
0080c300   Edma_Test_Start
0080a96c   Exception_service_routine
0080fea0   HOSTclose
0080ee60   HOSTlseek
0080f260   HOSTopen
0080f960   HOSTread
0080e0a0   HOSTrename
0080fa20   HOSTunlink
0080fae0   HOSTwrite
008010e0   IDMA_copy
008059e4   IDMA_wait
00804ba0   KeyStone_CIC_EXC_handler
00803a74   KeyStone_CIC_exception_events_mapping
0080598c   KeyStone_CorePac_AID_map
00805d80   KeyStone_DDR_ECC_INT_enable
00805d94   KeyStone_DDR_ECC_init
008066a0   KeyStone_DDR_PLL_init
00805cc0   KeyStone_DDR_clock_phase_init
00805f34   KeyStone_DDR_full_leveling
00807e38   KeyStone_DDR_init
00805d34   KeyStone_DDR_latch_leveling_configuration
00805fcc   KeyStone_DDR_read_incremental_leveling
00805300   KeyStone_EXC_external
00804060   KeyStone_Exception_cfg
00809ea8   KeyStone_MPAX_seg_setup
00803948   KeyStone_MPU_MPPA_modify
0080372c   KeyStone_MPU_interrupts_enable
00803400   KeyStone_MPU_range_setup
00803484   KeyStone_MPU_setup
008033b0   KeyStone_MSMC_MP_interrupt_en
008032c0   KeyStone_MSMC_protection_exception_handler
00803284   KeyStone_PrivID_Remap
008031a0   KeyStone_SES_MPAX_setup
008030d4   KeyStone_SL2_EDC_enable
00802d74   KeyStone_SL2_EDC_handler
00802d28   KeyStone_SL2_EDC_interrupt_en
00802c48   KeyStone_SMS_MPAX_setup
0080a0a0   KeyStone_XMC_MPAX_setup
00802bb4   KeyStone_disable_PSC_Power_Domain
00802b28   KeyStone_disable_PSC_module
00802a6c   KeyStone_enable_PSC_module
008026c0   KeyStone_main_PLL_init
008025ac   KeyStone_peripherals_MPU_excepiton_handler
00802484   KeyStone_peripherals_MPU_fault_status
008023ec   KeyStone_print_device_info
008017c0   L1D_memory_protection_cfg
00801fec   L1P_EDC_setup
00801e44   L1P_ED_handler
008015ec   L1P_memory_protection_cfg
00801c84   L1_MPPA_setup
00801960   L1_cache_protection
00814978   L2CacheSize
00814934   LL2_EDC_DMA_err_str
00814938   LL2_EDC_L1D_err_str
0081493c   LL2_EDC_L1P_err_str
00801360   LL2_EDC_handler
008012ac   LL2_EDC_scrub
00801140   LL2_EDC_setup
00814930   LL2_EDC_victim_err_str
00800f20   LL2_MPPA_setup
00800c20   LL2_Memory_Protection_cfg
00814914   MPU0_Regs
00814918   MPU1_Regs
0081491c   MPU2_Regs
00814920   MPU3_Regs
008144b0   MPU_Regs
00810620   MemCopy8
0080a800   Nested_Exception_service_routine
00814590   Ns_str
00814530   Peri_MPU_err_type_str
008008e8   Reset_Timer
00800bf0   Service_Watchdog
008060a4   TCI6614_EVM_DDR_Init
00800b70   TN_MPU5_constant
00800ae0   TSC_delay_ms
00800a68   TSC_delay_us
00800a28   TSC_init
0080090c   Timer64_Init
00808be0   Timer_ISR
00814890   XMC_regs
00814770   __CIOBUF_
00814e9c   __TI_CINIT_Base
00814ec4   __TI_CINIT_Limit
00814e88   __TI_Handler_Table_Base
00814e94   __TI_Handler_Table_Limit
UNDEFED    __TI_INITARRAY_Base
UNDEFED    __TI_INITARRAY_Limit
00813850   __TI_STACK_END
00001000   __TI_STACK_SIZE
00814890   __TI_STATIC_BASE
00000800   __TI_SYSMEM_SIZE
UNDEFED    __TI_TLS_INIT_Base
UNDEFED    __TI_TLS_INIT_Limit
00000001   __TI_args_main
008109a0   __TI_cpp_init
00810e00   __TI_decompress_none
00810e20   __TI_decompress_rle24
0081457c   __TI_enable_exit_profile_output
ffffffff   __TI_pprof_out_hndl
ffffffff   __TI_prof_data_size
ffffffff   __TI_prof_data_start
0080fde0   __TI_tls_init
0080f5e0   __TI_zero_init
ffffffff   __binit__
00809240   __c6xabi_divd
0080c860   __c6xabi_divf
0080fba0   __c6xabi_divu
0080e3e0   __c6xabi_divul
0080cfe0   __c6xabi_divull
008106a0   __c6xabi_fixdu
00810720   __c6xabi_fixfu
00810a00   __c6xabi_frcmpyd_div
00810c20   __c6xabi_isinf
008107a0   __c6xabi_llshl
00810a60   __c6xabi_llshru
00810d60   __c6xabi_negll
00810ca0   __c6xabi_strasgi_64plus
ffffffff   __c_args__
0080fba0   __divu
00810ca0   __strasgi_64plus
00810ce0   _args_main
0080ef60   _auto_init_elf
00810820   _c_int00
0080ff40   _cleanup
00814574   _cleanup_ptr
0080eb00   _closefile
00812638   _ctypes_
0080fc60   _doflush
00814578   _dtors_ptr
008143f4   _ft_end
00814050   _ftable
00814598   _lock
00810120   _minit
00810d80   _nop
0080ace0   _printfi
00812850   _stack
00810ac0   _subcull
00813850   _sys_memory
008145a0   _tmpnams
0081459c   _unlock
0080f060   _wrt_ok
00810de0   abort
0080f420   atoi
ffffffff   binit
00814898   boot_cfg_regs
008144d0   bus_err_stat_str
008008b0   calc_cycle_measure_overhead
0080f500   close
0080f160   copy_in
00814510   coreEnableMaskPattern
0081496c   coreInfo
1081f280   coreTestInfo
008148b0   cpIntc0Regs
008148b4   cpIntc1Regs
00814928   cycle_measure_overhead
008143a8   dmaEnableMaskPattern
00814980   dstAddr
1081f000   edmaTestInfo
00800428   edma_Init
008003f0   edma_TC_priority_cfg
008003b8   edma_channel_TC_cfg
00814548   edma_sys_event_num
00814950   enableMaskLoop
008146e0   exception_record
0080fd20   exit
0080d8c0   fputc
0080b960   fputs
0080cd60   free
0080ed40   fseek
008144f0   gCIC_EXC_EN_MASK
00814944   gCIC_EXC_out_num
008148bc   gEDMACC0Regs
008148c0   gEDMACC1Regs
008148c4   gEDMACC2Regs
00814558   gEDMACCRegs
008148c8   gEDMA_TC_0_0_Regs
008148cc   gEDMA_TC_0_1_Regs
008148d0   gEDMA_TC_1_0_Regs
008148d4   gEDMA_TC_1_1_Regs
008148d8   gEDMA_TC_1_2_Regs
008148dc   gEDMA_TC_1_3_Regs
008148e0   gEDMA_TC_2_0_Regs
008148e4   gEDMA_TC_2_1_Regs
008148e8   gEDMA_TC_2_2_Regs
008148ec   gEDMA_TC_2_3_Regs
00814438   gEDMA_TC_Regs
008148a8   gpioRegs
008143f8   gstruMpuAddrRange
00814940   guwIntcCICExcEvtIdx
00814460   internal_exception_str
00809e2c   lock_mem_prot_regs
00810300   lseek
0080f6c0   ltoa
008088b4   main
0080e700   malloc
00814748   mem_prot_key
00810b20   memccpy
008103a0   memcpy
00800200   memory_protection_exception_handler
0080f7a0   memset
008148a4   msmcRegs
0081489c   pllc_regs
0080f880   printf
0081494c   priorityLoop
00814568   priorityPattern
008148a0   pscRegs
00810d20   puts
008108a0   readmsg
1081f480   readyFlag
00810920   remove
00814974   repeatCount
008082a4   restartDSPCore
008080f8   restartEDMA
0080dce0   setvbuf
00814970   size
0081497c   srcAddr
00814958   srcDstSwap
00814968   start_TSC
008080cc   swapDSPCoreAddress
008080a0   swapEDMAAddress
00814948   testCaseCnt
00814348   testCases
00814954   testCount
008148f0   timer0Regs
008148f4   timer1Regs
008148f8   timer2Regs
008148fc   timer3Regs
00814900   timer4Regs
00814904   timer5Regs
00814908   timer6Regs
0081490c   timer7Regs
00814910   timer8Regs
00814488   timerRegs
00814758   uiEdma_host_event_num
00814964   uiIntCnt
0081492c   uiLL2_scrub_addr
00814960   uiSysIntNoIprCnt
0081495c   uiUnexpectIntCnt
00810920   unlink
00809dc0   unlock_mem_prot_regs
00800000   vectors
00810580   write
00810b80   writemsg


GLOBAL SYMBOLS: SORTED BY Symbol Address 

address    name
--------   ----
00000001   __TI_args_main
00000800   __TI_SYSMEM_SIZE
00001000   __TI_STACK_SIZE
00800000   vectors
00800200   memory_protection_exception_handler
008003b8   edma_channel_TC_cfg
008003f0   edma_TC_priority_cfg
00800428   edma_Init
008008b0   calc_cycle_measure_overhead
008008e8   Reset_Timer
0080090c   Timer64_Init
00800a28   TSC_init
00800a68   TSC_delay_us
00800ae0   TSC_delay_ms
00800b70   TN_MPU5_constant
00800bf0   Service_Watchdog
00800c20   LL2_Memory_Protection_cfg
00800f20   LL2_MPPA_setup
008010e0   IDMA_copy
00801140   LL2_EDC_setup
008012ac   LL2_EDC_scrub
00801360   LL2_EDC_handler
008015ec   L1P_memory_protection_cfg
008017c0   L1D_memory_protection_cfg
00801960   L1_cache_protection
00801c84   L1_MPPA_setup
00801e44   L1P_ED_handler
00801fec   L1P_EDC_setup
008023ec   KeyStone_print_device_info
00802484   KeyStone_peripherals_MPU_fault_status
008025ac   KeyStone_peripherals_MPU_excepiton_handler
008026c0   KeyStone_main_PLL_init
00802a6c   KeyStone_enable_PSC_module
00802b28   KeyStone_disable_PSC_module
00802bb4   KeyStone_disable_PSC_Power_Domain
00802c48   KeyStone_SMS_MPAX_setup
00802d28   KeyStone_SL2_EDC_interrupt_en
00802d74   KeyStone_SL2_EDC_handler
008030d4   KeyStone_SL2_EDC_enable
008031a0   KeyStone_SES_MPAX_setup
00803284   KeyStone_PrivID_Remap
008032c0   KeyStone_MSMC_protection_exception_handler
008033b0   KeyStone_MSMC_MP_interrupt_en
00803400   KeyStone_MPU_range_setup
00803484   KeyStone_MPU_setup
0080372c   KeyStone_MPU_interrupts_enable
00803948   KeyStone_MPU_MPPA_modify
00803a74   KeyStone_CIC_exception_events_mapping
00804060   KeyStone_Exception_cfg
008041e4   EDMA_CC_error_handler
00804420   EDMA_TC_error_handler
008045c8   EDMA_error_handler
00804ba0   KeyStone_CIC_EXC_handler
008051ec   Bus_error_handler
00805300   KeyStone_EXC_external
0080598c   KeyStone_CorePac_AID_map
008059e4   IDMA_wait
00805a24   EXC_swgen
00805a34   EXC_internal
00805b44   EXC_NMI
00805b54   EDMA_wait
00805be0   EDMA_copy
00805cc0   KeyStone_DDR_clock_phase_init
00805d34   KeyStone_DDR_latch_leveling_configuration
00805d80   KeyStone_DDR_ECC_INT_enable
00805d94   KeyStone_DDR_ECC_init
00805f34   KeyStone_DDR_full_leveling
00805fcc   KeyStone_DDR_read_incremental_leveling
008060a4   TCI6614_EVM_DDR_Init
008066a0   KeyStone_DDR_PLL_init
00806824   C6670_EVM_DDR_Init
00806da4   C6678_EVM_DDR_Init
00807360   Dual_Nyquist_EVM_DDR_Init
00807ac0   DDR_Fill_Test
00807c80   DDR_Address_Test
00807e38   KeyStone_DDR_init
008080a0   swapEDMAAddress
008080cc   swapDSPCoreAddress
008080f8   restartEDMA
008082a4   restartDSPCore
00808410   EDMA_init_for_mem_share
00808584   ConfigureTest
0080880c   EDMA_pri_set
008088b4   main
00808be0   Timer_ISR
00809240   __c6xabi_divd
00809dc0   unlock_mem_prot_regs
00809e2c   lock_mem_prot_regs
00809ea8   KeyStone_MPAX_seg_setup
0080a0a0   KeyStone_XMC_MPAX_setup
0080a2e0   DSP_core_mem_share_Test
0080a74c   DSP_Core_Test_Start
0080a800   Nested_Exception_service_routine
0080a96c   Exception_service_routine
0080ace0   _printfi
0080b5a0   EDMA_ISR
0080b960   fputs
0080c300   Edma_Test_Start
0080c860   __c6xabi_divf
0080cd60   free
0080cfe0   __c6xabi_divull
0080d8c0   fputc
0080dce0   setvbuf
0080e0a0   HOSTrename
0080e240   EDMA_Timer_Interrupts_Init
0080e2a0   CP_INTC_Init_EDMA
0080e3e0   __c6xabi_divul
0080e700   malloc
0080eb00   _closefile
0080ed40   fseek
0080ee60   HOSTlseek
0080ef60   _auto_init_elf
0080f060   _wrt_ok
0080f160   copy_in
0080f260   HOSTopen
0080f420   atoi
0080f500   close
0080f5e0   __TI_zero_init
0080f6c0   ltoa
0080f7a0   memset
0080f880   printf
0080f960   HOSTread
0080fa20   HOSTunlink
0080fae0   HOSTwrite
0080fba0   __c6xabi_divu
0080fba0   __divu
0080fc60   _doflush
0080fd20   exit
0080fde0   __TI_tls_init
0080fea0   HOSTclose
0080ff40   _cleanup
00810120   _minit
00810300   lseek
008103a0   memcpy
00810580   write
00810620   MemCopy8
008106a0   __c6xabi_fixdu
00810720   __c6xabi_fixfu
008107a0   __c6xabi_llshl
00810820   _c_int00
008108a0   readmsg
00810920   remove
00810920   unlink
008109a0   __TI_cpp_init
00810a00   __c6xabi_frcmpyd_div
00810a60   __c6xabi_llshru
00810ac0   _subcull
00810b20   memccpy
00810b80   writemsg
00810bd8   C$$IO$$
00810c20   __c6xabi_isinf
00810ca0   __c6xabi_strasgi_64plus
00810ca0   __strasgi_64plus
00810ce0   _args_main
00810d20   puts
00810d60   __c6xabi_negll
00810d80   _nop
00810de0   C$$EXIT
00810de0   abort
00810e00   __TI_decompress_none
00810e20   __TI_decompress_rle24
00812638   _ctypes_
00812850   _stack
00813850   __TI_STACK_END
00813850   _sys_memory
00814050   _ftable
00814348   testCases
008143a8   dmaEnableMaskPattern
008143f4   _ft_end
008143f8   gstruMpuAddrRange
00814438   gEDMA_TC_Regs
00814460   internal_exception_str
00814488   timerRegs
008144b0   MPU_Regs
008144d0   bus_err_stat_str
008144f0   gCIC_EXC_EN_MASK
00814510   coreEnableMaskPattern
00814530   Peri_MPU_err_type_str
00814548   edma_sys_event_num
00814558   gEDMACCRegs
00814568   priorityPattern
00814574   _cleanup_ptr
00814578   _dtors_ptr
0081457c   __TI_enable_exit_profile_output
00814590   Ns_str
00814598   _lock
0081459c   _unlock
008145a0   _tmpnams
008146e0   exception_record
00814748   mem_prot_key
00814758   uiEdma_host_event_num
00814770   __CIOBUF_
00814890   XMC_regs
00814890   __TI_STATIC_BASE
00814894   CGEM_regs
00814898   boot_cfg_regs
0081489c   pllc_regs
008148a0   pscRegs
008148a4   msmcRegs
008148a8   gpioRegs
008148ac   DDR_Regs
008148b0   cpIntc0Regs
008148b4   cpIntc1Regs
008148b8   CIC_Regs
008148bc   gEDMACC0Regs
008148c0   gEDMACC1Regs
008148c4   gEDMACC2Regs
008148c8   gEDMA_TC_0_0_Regs
008148cc   gEDMA_TC_0_1_Regs
008148d0   gEDMA_TC_1_0_Regs
008148d4   gEDMA_TC_1_1_Regs
008148d8   gEDMA_TC_1_2_Regs
008148dc   gEDMA_TC_1_3_Regs
008148e0   gEDMA_TC_2_0_Regs
008148e4   gEDMA_TC_2_1_Regs
008148e8   gEDMA_TC_2_2_Regs
008148ec   gEDMA_TC_2_3_Regs
008148f0   timer0Regs
008148f4   timer1Regs
008148f8   timer2Regs
008148fc   timer3Regs
00814900   timer4Regs
00814904   timer5Regs
00814908   timer6Regs
0081490c   timer7Regs
00814910   timer8Regs
00814914   MPU0_Regs
00814918   MPU1_Regs
0081491c   MPU2_Regs
00814920   MPU3_Regs
00814924   DSP_Core_Clock_KHz
00814928   cycle_measure_overhead
0081492c   uiLL2_scrub_addr
00814930   LL2_EDC_victim_err_str
00814934   LL2_EDC_DMA_err_str
00814938   LL2_EDC_L1D_err_str
0081493c   LL2_EDC_L1P_err_str
00814940   guwIntcCICExcEvtIdx
00814944   gCIC_EXC_out_num
00814948   testCaseCnt
0081494c   priorityLoop
00814950   enableMaskLoop
00814954   testCount
00814958   srcDstSwap
0081495c   uiUnexpectIntCnt
00814960   uiSysIntNoIprCnt
00814964   uiIntCnt
00814968   start_TSC
0081496c   coreInfo
00814970   size
00814974   repeatCount
00814978   L2CacheSize
0081497c   srcAddr
00814980   dstAddr
00814e88   __TI_Handler_Table_Base
00814e94   __TI_Handler_Table_Limit
00814e9c   __TI_CINIT_Base
00814ec4   __TI_CINIT_Limit
1081f000   edmaTestInfo
1081f280   coreTestInfo
1081f480   readyFlag
ffffffff   __TI_pprof_out_hndl
ffffffff   __TI_prof_data_size
ffffffff   __TI_prof_data_start
ffffffff   __binit__
ffffffff   __c_args__
ffffffff   binit
UNDEFED    __TI_INITARRAY_Base
UNDEFED    __TI_INITARRAY_Limit
UNDEFED    __TI_TLS_INIT_Base
UNDEFED    __TI_TLS_INIT_Limit

[271 symbols]
